:040000008A11112828
:10000800FE00030EF1000408F2000A08F300831250
:1000180003137F08F4008A11BD2A8A111328F801F6
:100028008313393084004C308A11782383018A1174
:100038001D288B010730831203139F0001308500B0
:1000480001308316031385008312031386010230DF
:1000580083160313860006308312031381008B1660
:1000680004308316031381007D3083120313B50017
:100078003508CC00C001BF017810B901BA01C2012E
:10008800C301C101BB017811BC01BD010030A00052
:100098000030A1000830A2000030A30044308A11CB
:1000A8002E238A11F810F8118312031306108A11EF
:1000B80051238A118B178312031385143F08053ABD
:1000C8000319781C6B288A1147218A11781083122A
:1000D80003138C1E88281930B5003508BE0004307B
:1000E800B5003508BB008C1298187C28181D832889
:1000F800981C802818121816181D88288428781526
:100108001A08B5003508BC00BE080319BD01781DE2
:100118009E2808303D0203189E2878113C08B50037
:100128003D08443E84003508831380000130B50043
:100138003508BD0708303D02031CCE28B701B801B9
:10014800073038020318C3283808443E8400831354
:100158000008B5003508F5003808013E8A11652306
:100168008A11831203133707B6003608B700013027
:10017800B5003508B80707303802031CA8284B0813
:100188003706031DCD2844080C3A031DCD28F81462
:10019800CE28BD01F81C6228F8104508C13A031D95
:1001A800DA28C230B5003508C600F8154508023A05
:1001B800031DF3283908B5003508C6003A08B5000C
:1001C8003508C7004208B5003508C8004308B5001F
:1001D8003508C9004108B5003508CA00F815F81DEA
:1001E8004529F811B701B801073038020318172953
:1001F8003808443E840083130008B5003508F5002C
:100208003808013E8A1165238A11831203133707C0
:10021800B6003608B7000130B5003508B807073012
:100228003802031CFC283708B5003508CB00061433
:10023800B80108303802031844290430B5003508DD
:10024800BB003808443E8400831300089900193025
:10025800B5003508BE008316031398183829831291
:100268000313BE08031D2F298312BE08031944294E
:100278000130B5003508B80708303802031C2129B9
:100288000610BD0162288A11F9218A110038031964
:1002980008008A113B228A1183120313A70027083A
:1002A800B2008A113B228A1183120313A700270880
:1002B800B1008A113B228A1183120313A700270871
:1002C800B4008A113B228A1183120313A70027085E
:1002D800B3008A113B228A1183120313A70027084F
:1002E800AB0031083207A70034082707A8003308F5
:1002F8002807A9002908AC002B082C06031D0800B4
:10030800B41F8E2934087F39A7002708B400C1011B
:10031800C10A8F29C1013108A700A8013208A90024
:10032800AA012908AA00A90127082904AD0028085C
:100338002A04AE003308A700A8013408A900AA01BE
:100348002908AA00A90127082904AF0028082A04B7
:10035800B0000A30A0000030A1002E08A301A307B6
:100368002D08A201A2078A117D228A118312031384
:100378002008A7002708B9000A30A0000030A10013
:100388002E08A301A3072D08A201A2078A11F822AB
:100398008A11831203132008A7002708BA000A301D
:1003A800A0000030A1003008A301A3072F08A20174
:1003B800A2078A117D228A11831203132008A7003D
:1003C8002708C2000A30A0000030A1003008A301AD
:1003D800A3072F08A201A2078A11F8228312031388
:1003E8002008A7002708C3000800F6018316031396
:1003F8000510831203130510F930F5000000F50B02
:10040800022A062A00008316031305148312031315
:1004180005140518112A760808006430F5007508D7
:10042800F7001B2AF70803191D2A0130F7020518DF
:10043800162A0518212AF601F60A6430F50075080F
:10044800F700282A0130F70205182D2AF708031D9E
:10045800262A6430F5007508F700342A0130F702BF
:10046800051C392AF708031D322A7608080083126A
:100478000313A201A001A00A0930200203187B2A55
:100488006430F5007508A1004B2A0130A102051857
:10049800502AA108031D492A0B30F500F50B522AF2
:1004A8000000831203132208F5007507F60076088A
:1004B800A200051C622A22080138642A2208FE3993
:1004C800F5007508A2006430F5007508A1006E2AD1
:1004D8000130A102051C732AA108031D6C2A0130F2
:1004E800F5007508A00709302002031C442A2208D9
:1004F800080083120313A501A6012108200403198B
:10050800B62AA401A40AA11B952A01300310A00D44
:10051800A10DFF3E031D8A2A0130F5007508A407C6
:10052800872A01300310A50DA60DFF3E031D962A4C
:1005380021082302031DA22A20082202031CAB2A39
:100548002008A2022108031CA303A30225140130DA
:100558000310A10CA00CFF3E031DAC2A0130A4021D
:10056800031D952A2608A101A1072508A001A007B7
:1005780008000B1DED2A0B11063081000130CC025A
:10058800CC08031DD82A7D30F0007008CC00043058
:10059800F0007008C0000130F0007008BF070A3092
:1005A8003F020318BF01781440080319DF2A0130FD
:1005B800C0020515E02A05113B080319E72A013096
:1005C800BB028515E82A85113E080319ED2A01307A
:1005D800BE027408FF0073088A0072088400710E56
:1005E8008300FE0E7E0E09008312031321082004E7
:1005F8000319272BF601F60AA11B0E2B0130031055
:10060800A00DA10DFF3E031D032B0130F500750859
:10061800F607002B21082302031D142B20082202B1
:10062800031C1C2B2008A2022108031CA303A302FD
:1006380001300310A10CA00CFF3E031D1D2B01303F
:10064800F602031D0E2B2308A101A1072208A00111
:10065800A0070800F6007608F5007508F7000130D5
:1006680083120313A2020030031CA303A302FF306A
:100678002306031D412BFF302206031908008312AD
:1006880003132008F5007708840075088313800099
:100698000130F5007508F707332B83160313181577
:1006A8000C30990018128312031398171813831625
:1006B80003131813831203131816831603139816BB
:1006C800080083120313A100A001211C6F2B7508D9
:1006D800F6007608A0070310F50D0310A10CA10879
:1006E800031D692B2008080064008001840A0406A1
:0806F800031900340406792BFC
:02400E0061FF50
:00000001FF
